:020000040000FA
:0400000003303A2867
:08000800A000030EA100831209
:1000100005191128831601178312B2308100B0012F
:100020002C2883160113831203140B190310A80D37
:10003000A90DAA0DAB0DAC0DAC16FF302C02031DA3
:100040002C28FA302B02031D2C2831152A08AF006A
:100050002908AE002808AD008B100B11210E83007B
:06006000A00E200E0900B5
:0C007400203084008001840A6030040207
:10008000031C3C2897218316FF23900083128316BC
:100090000C3085058701831285018701073099009F
:1000A0000030831691009F008312C83083168100B0
:1000B000831231309000003083168C008312103090
:1000C0008B00BC1B6928851969286400851D65287B
:1000D000E021D82181018E018F010B118B100B10B3
:1000E0008C018B17812031198D20B30B7F280310D1
:1000F00085190314B90DF0303902031912210522B4
:10010000722864003210B00A301F8C28AC01AB0199
:10011000AA01A901A801B001080031110130B700FE
:100120008B132030370783169B001C141A08831288
:10013000A4001030370783169B001C141A08831282
:10014000A300A6000230A6060030370783169B00E6
:100150001C141A088312A200A7000130A7068B17EF
:10016000321CB82822090339A200A309A409A50951
:1001700024082F02031D0C2923082E02031D0C291D
:1001800022082D02031D0C2901303702031DCD2842
:100190003D18CD283D143E14AC2102303702031D1A
:1001A000D628BD18D628BD143E14B021033037021E
:1001B000031DDF283D19DF283D153E14B42104300E
:1001C0003702031DE828BD19E828BD153E14B821E3
:1001D00005303702031DF1283D1AF1283D163E1463
:1001E000BC2106303702031DFA28BD1AFA28BD16B5
:1001F0003E14BD2107303702031D03293D1B03298F
:100200003D173E14BE2108303702031D0C29BD1BCB
:100210000C29BD173E14BF21B70A05303702031859
:10022000080090280130B600B300B400B500B70054
:1002300085018701B1138120B30B4A290310851969
:100240000314B90DF030390203197129B40B4A298E
:10025000013037020319C021023037020319C421CB
:10026000033037020319C821043037020319D021A3
:10027000053037020319D421063037020319D5217E
:10028000073037020319D621083037020319D72166
:100290009630B400311D1B293111321C54292D090F
:1002A0000339AD00AE09AF092F1C1B298E018F0148
:1002B0000C1C1B290C102E1E1B298B1320303707FA
:1002C000BB002F08BA00842110303707BB002E086E
:1002D000BA00842100303707BB002D08BA00842102
:1002E0008B1785018701B70AB60105303702031C59
:1002F0001B29D82108003E1C08003E101030BB000E
:100300003D08BA00842108008B133A0883161C1597
:100310009A003B089B0055309D00AA309D009C141C
:1003200064009C1890291C1183128B1708008316F7
:1003300000309B001C141A088312BC008316103076
:100340009B001C141A088312BD00FF30D000D41586
:10035000D515D615D71508000330D204BD100800F6
:100360000330D2043D1008000C30D204BD11080047
:100370000C30D2043D1108000800080008000800F5
:100380000508023A850008000508013A85000800C2
:100390000C308316850083120508203A850008007A
:1003A0000508103A85000800080008000800080049
:1003B0003D08D200031D08000530BD00D200080032
:1003C000B601B301B4013C1CE829BC01BC14EA2904
:1003D000BC013C143C08B6006400EE29EF29F0296A
:1003E000F129F229B41B8514B41F8510B30BEC2935
:1003F000B40BEC290310B60CB608031DEC29003031
:10040000BB003C08BA00842108008F0803190800CB
:100410008F01D00FA62AD00A02305205031D1F2AD1
:10042000541D152AD40154162D2AD41D1A2AD4017C
:1004300054162D2A541E2D2AD401D4142D2AD41C2E
:10044000242AD40154152D2A541D292AD401D41547
:100450002D2A541E2D2AD401541501305205031D96
:10046000402A551D362AD50155164E2AD51D3B2A40
:10047000D50155164E2A551E4E2AD501D5144E2AA1
:10048000D51C452AD50155154E2A551D4A2AD50198
:10049000D5154E2A551E4E2AD50155150830BC18C3
:1004A0000A305205031D632A561D592AD6015616D5
:1004B000712AD61D5E2AD6015616712A561E712A39
:1004C000D601D614712AD61C682AD6015615712A6F
:1004D000561D6D2AD601D615712A561E712AD601CF
:1004E00056150430BC1806305205031D862A571DC8
:1004F0007C2AD7015716942AD71D812AD70157166F
:10050000942A571E942AD701D714942AD71C8B2AD1
:10051000D7015715942A571D902AD701D715942A29
:10052000571E942AD7015715BC1C9F2AD21C9F2AFC
:10053000D51C9F2A3C30831685008312A32A0C30D9
:100540008316850083127B213D08D2005008D1001C
:100550000C305405031D85100C305505031D051086
:100560000C305605031D85120C305705031D05126E
:1005700051080E020318D02A12305405031D8514A9
:1005800012305505031D051412305605031D85163E
:1005900012305705031D0516FF30500203190800DD
:1005A0008F08031D0800812051080E02031CD02A69
:1005B00018305405031D851006305405031D85149D
:1005C00018305505031D051006305505031D05148B
:1005D00018305605031D851206305605031D851675
:1005E00018305705031D051206305705031D051663
:0205F000080001
:084000000200030006000600A7
:02400E00CC01E3
:10420000010078007A007C007E007B0079007F004E
:104210007D007A0078007E007C00FF00FF00FF0038
:104220000000F200F600FA00FE00F200F600FA00CC
:10423000FE00F200F600FA00FE00FF00FF00FF00A3
:10424000010005000500050005000900090009003E
:1042500009000D000D000D000D00FF00FF00FF0024
:10426000FF00FF00FF00FF00FF00FF00FF00FF0056
:10427000FF00FF00FF00FF00FF00FF00FF00FF0046
:10428000FF00FF00FF00FF00FF00FF00FF00FF0036
:10429000FF00FF00FF00FF00FF00FF00FF00FF0026
:1042A000FF00FF00FF00FF00FF00FF00FF00FF0016
:1042B000FF00FF00FF00FF00FF00FF00FF00FF0006
:1042C000FF00FF00FF00FF00FF00FF00FF00FF00F6
:1042D000FF00FF00FF00FF00FF00FF00FF00FF00E6
:1042E000FF00FF00FF00FF00FF00FF00FF00FF00D6
:1042F000FF00FF00FF00FF00FF00FF00FF00DD00E8
:00000001FF
